:020000000147B6
:020003000147B3
:02000B000125CD
:02001B000136AC
:180023000147C0E0C0D0D24085088A85098CD0D0D0E032C0E0C0D085D3
:18003B000A8B850B8DD241D0D0D0E03275A80075D00075812FE4787F04
:18005300F6D8FD75880075A80A758911D2AFC249C248751000751100F6
:18006B00751800751900750C33750D3301793049031200BB30480312A9
:1800830000D1D2B020B015204912D249D2B120B105751001019C751096
:18009B0002751201D2B320B315204812D248D2B220B205751801800356
:1800B300751802751A000179D2B030B00DC28CC240751100D2B4C249C7
:1800CB0001D01200E722D2B330B30DC28EC241751900D2B5C24801E663
:1800E300120112227911B7000201FE2040022111C28CC240A812E510E9
:1800FB0012013F7508007509EF85088A85098CD28C751102C2B4227989
:1801130019B70002212B204102213EC28EC241A81AE51812013FC2418D
:18012B00750A00750BEF850A8B850B8DD28E751902C2B522B80020C373
:18014300B40105E50C03214EE50C23F50C540FF5F0C2AFE59054F045BB
:18015B00F0F590D2AF2180C3B40105E50D03216EE50D23F50D54F0F5A4
:0E017300F0C2AFE590540F45F0F590D2AF22E8
:00000001FF
